:100000000C9473000C949B000C949B000C949B002C
:100010000C949B000C9418080C949B000C949B006F
:100020000C949B000C949B000C949B000C949B00E4
:100030000C949B000C949B000C949B000C949B00D4
:100040000C947D050C949B000C948F040C94690413
:100050000C949B000C949B000C949B000C949B00B4
:100060000C94C7050C949B00980C9A0C9C0C9E0C4D
:10007000A00CA20CA40CA60CD80CDB0CDE0CD50C2E
:10008000E10CE40CF50CF50C000000002400270046
:100090002A0000000000250028002B0000000000BE
:1000A00023002600290004040404040404040202BA
:1000B00002020202030303030303010204081020E7
:1000C00040800102040810200102040810200000F2
:1000D0000008000201000003040700000000000007
:1000E0000000E822982211241FBECFEFD8E0DEBF27
:1000F000CDBF24E0AEE4B2E001C01D92AB3CB2073C
:10010000E1F712E0A0E0B1E0ECE3F2E502C0059017
:100110000D92AE34B107D9F710E0C2E7D0E004C0C9
:100120002197FE010E946525C137D107C9F70E94BA
:1001300056150C9411290C9400000895CF92DF926B
:10014000EF92FF920F931F93CF93DF936C017A018D
:100150008B01C0E0D0E0CE15DF0589F0D8016D91AC
:100160008D01D601ED91FC910190F081E02DC60149
:100170000995892B11F47E0102C02196ECCFC701AD
:10018000DF91CF911F910F91FF90EF90DF90CF9073
:100190000895FC01918D828D981761F0828DDF01A9
:1001A000A80FB11D5D968C91928D9F5F9F73928F6A
:1001B00090E008958FEF9FEF0895FC01918D828D5F
:1001C000981731F0828DE80FF11D858D90E008952C
:1001D0008FEF9FEF0895FC01918D228D892F90E084
:1001E000805C9F4F821B91098F73992708958DE43E
:1001F00093E00E94EB0021E0892B09F420E0822F9C
:100200000895FC01848DDF01A80FB11DA35ABF4FD3
:100210002C91848D90E001968F739927848FA68905
:10022000B7892C93A089B1898C9180648C93938D2C
:10023000848D981306C00288F389E02D80818F7D1C
:1002400080830895EF92FF920F931F93CF93DF93D4
:10025000EC0181E0888F9B8D8C8D981305C0E88917
:10026000F989808185FD24C0F62E0B8D10E00F5F8B
:100270001F4F0F731127E02E8C8DE8120CC00FB6A4
:1002800007FCFACFE889F989808185FFF5CFCE0197
:100290000E940101F1CF8B8DFE01E80FF11DE35AA1
:1002A000FF4FF0820B8FEA89FB898081806207C053
:1002B000EE89FF896083E889F98980818064808381
:1002C00081E090E0DF91CF911F910F91FF90EF902F
:1002D0000895CF93DF93EC01888D8823C9F0EA89D4
:1002E000FB89808185FD05C0A889B9898C9186FD2F
:1002F0000FC00FB607FCF5CF808185FFF2CFA8892C
:10030000B9898C9185FFEDCFCE010E940101E7CF25
:10031000DF91CF91089580E090E0892B29F00E9431
:10032000F70081110C9400000895833081F028F4C7
:10033000813099F08230A1F008958730A9F088309B
:10034000B9F08430D1F4809180008F7D03C080911A
:1003500080008F7780938000089584B58F7702C0E6
:1003600084B58F7D84BD08958091B0008F7703C0E0
:100370008091B0008F7D8093B0000895CF93DF937C
:10038000282F30E0F901E253FF4F8491F901E65440
:10039000FF4FD491F901EA55FF4FC491CC2391F05E
:1003A00081110E949501EC2FF0E0EE0FFF1FE45643
:1003B000FF4FA591B491EC91ED2381E090E021F401
:1003C00080E002C080E090E0DF91CF9108953FB7D8
:1003D000F8948091DC029091DD02A091DE02B09150
:1003E000DF0226B5A89B05C02F3F19F00196A11D7D
:1003F000B11D3FBFBA2FA92F982F8827820F911DBB
:10040000A11DB11DBC01CD0142E0660F771F881F01
:10041000991F4A95D1F7089585ED8093BC0080918E
:10042000BC0084FDFCCF1092280308954091B602D1
:10043000262F30E0240F311D21323105DCF42091CC
:1004400028032430C9F4FC0180E090E0861758F4BA
:100450003091B6022191DC01AC56BD4FA30FB11D06
:100460002C930196F3CF8091B602680F6093B60289
:1004700080E0089581E0089582E008950895E09174
:10048000E1028091E002E81730F4F0E0EE51FD4F18
:10049000808190E008958FEF9FEF08959091E102A1
:1004A0008091E002981750F4E92FF0E0EE51FD4FF3
:1004B000208130E09F5F9093E10202C02FEF3FEF79
:1004C000C90108958091E00290E02091E102821B31
:1004D00091090895CF92DF92EF92FF920F931F93AD
:1004E000CF93DF937C01262F972F8A0180912903D8
:1004F000882391F0C62FD72F6E01C40ED51ECC15C0
:10050000DD0571F06991D701ED91FC910190F081C9
:10051000E02DC7010995F3CF642F822F0E941602A8
:10052000C801DF91CF911F910F91FF90EF90DF9065
:10053000CF900895CF93DF931F92CDB7DEB7698335
:10054000209129032223D1F020914C03203240F046
:1005500021E030E0FC013383228380E090E015C08D
:1005600080912A03E82FF0E0E55DFC4F99819083AC
:100570008F5F80932A0380934C0305C061E0CE0116
:1005800001960E94160281E090E00F90DF91CF91DA
:1005900008950E94F328DF92EF92FF920F931F932A
:1005A000CF93DF9300D000D0CDB7DEB749835A8315
:1005B0006B837C837C018E010F5F1F4F84E0D82EFC
:1005C000D00EF80161918F01C7010E94B524FFEFA1
:1005D000EF1AFF0AD012F5CF0F900F900F900F90E7
:1005E000DF91CF911F910F91FF90EF90DF900895D1
:1005F000FC0180819181009711F00C940B2460E044
:1006000070E0CB0108950F931F93CF93DF938C017C
:10061000EB01FC01808191810097B1F068817981C3
:100620006115710579F0428153812C813D8142171A
:10063000530740F00E940A298C819D81F80195831F
:10064000848313C00E94912788819981F801918346
:1006500080838A819B81938382838C819D81958312
:100660008483198218821B821A821D821C82DF9168
:10067000CF911F910F9108950F931F93CF93DF9305
:10068000EC0188819981009729F02A813B81261706
:10069000370788F48B016F5F7F4F0E9429280097EE
:1006A00061F0998388831B830A832C813D81232BEE
:1006B00011F4FC01108281E001C080E0DF91CF9154
:1006C0001F910F910895EF92FF920F931F93CF9375
:1006D000DF93FC01248135816115710511F480E0FF
:1006E00019C041155105A9F07B01EC018A01020FE7
:1006F000131FB8010E943C03882389F328813981A4
:100700008C819D81B701820F931F0E940A291D834E
:100710000C8381E0DF91CF911F910F91FF90EF90BB
:100720000895CF93DF93EC0188819981009711F0B0
:100730000E949127198218821D821C821B821A82B4
:10074000DF91CF910895EF92FF920F931F93CF9374
:10075000DF93EC017B018A01BA010E943C03811105
:1007600004C0CE010E94910307C01D830C83B70112
:10077000888199810E940A29CE01DF91CF911F9132
:100780000F91FF90EF900895CF93DF93EC016115E7
:10079000710559F0FB0101900020E9F73197AF0195
:1007A000461B570B0E94A30302C00E949103CE0177
:1007B000DF91CF910895CF93DF93EC01FB01861772
:1007C000970761F0608171816115710529F044819D
:1007D00055810E94A30302C00E949103CE01DF91C4
:1007E000CF910895FC01808191810C949127FC01A7
:1007F0001182108213821282158214826115710592
:1008000051F0FB0101900020E9F73197AF01461B41
:10081000570B0C94A3030895BF92CF92DF92EF92EF
:10082000FF920F931F93CF93DF937C016B018A019B
:10083000E9012417350720F4812F8901C42FD82F0F
:1008400067E871E0C7010E94F703D60114968D9105
:100850009C91159708171907D0F48C179D0708F479
:10086000EC01D601ED91FC911197EC0FFD1FB080CA
:1008700010824D915C91BA01600F711FC7010E94F7
:10088000C403D601ED91FC91EC0FFD1FB082C701AE
:10089000DF91CF911F910F91FF90EF90DF90CF905C
:1008A000BF9008956115710579F0FB01019000205A
:1008B000E9F73197AF01461B570BDC01ED91FC9135
:1008C0000280F381E02D099480E090E008950C947B
:1008D00052041F920F920FB60F9211242F933F9341
:1008E0004F935F936F937F938F939F93AF93BF9338
:1008F000EF93FF938DE493E00E940101FF91EF914C
:10090000BF91AF919F918F917F916F915F914F9127
:100910003F912F910F900FBE0F901F9018951F922F
:100920000F920FB60F9211242F938F939F93EF93F3
:10093000FF93E0915D03F0915E038081E09163039A
:10094000F091640382FD12C09081809166038F5FF5
:100950008F7320916703821751F0E0916603F0E0F6
:10096000E35BFC4F958F8093660301C08081FF910C
:10097000EF919F918F912F910F900FBE0F901F902D
:1009800018951F93CF93DF93282F30E0F901E2539E
:10099000FF4F8491F901E654FF4FD491F901EA55D4
:1009A000FF4FC491CC23C9F0162F81110E949501ED
:1009B000EC2FF0E0EE0FFF1FEE56FF4FA591B49124
:1009C0008FB7F894111105C09C91ED2FE095E923A4
:1009D00002C0EC91ED2BEC938FBFDF91CF911F9173
:1009E0000895CF93DF93EC0160E08E810E94C104F3
:1009F00061E08E810E94C10460E08E810E94C1048A
:100A00008BE891E00197F1F7DF91CF910895CF93B3
:100A1000DF9390E0FC01E654FF4F2491FC01EA557E
:100A2000FF4F8491882361F190E0880F991FFC01AA
:100A3000E857FF4FC591D491FC01EE56FF4FA591A9
:100A4000B491611109C09FB7F894888120958223E1
:100A50008883EC912E230BC0623061F49FB7F89429
:100A60003881822F809583238883EC912E2B2C93C1
:100A70009FBF06C08FB7F894E8812E2B28838FBFC5
:100A8000DF91CF9108958F929F92AF92BF92CF92B4
:100A9000DF92EF92FF926B017C010E94E7014B0114
:100AA0005C01C114D104E104F104F1F00E94E701FA
:100AB000DC01CB0188199909AA09BB09883E93403A
:100AC000A105B10570F321E0C21AD108E108F108CF
:100AD00088EE880E83E0981EA11CB11CC114D104BD
:100AE000E104F10419F7DDCFFF90EF90DF90CF9094
:100AF000BF90AF909F908F9008951F920F920FB666
:100B00000F9211242F933F938F939F93AF93BF9393
:100B10008091520290915302A0915402B0915502DB
:100B20003091DB0223E0230F2D3720F40196A11D25
:100B3000B11D05C026E8230F0296A11DB11D20930B
:100B4000DB028093520290935302A0935402B0931D
:100B500055028091DC029091DD02A091DE02B091FD
:100B6000DF020196A11DB11D8093DC029093DD028E
:100B7000A093DE02B093DF02BF91AF919F918F915E
:100B80003F912F910F900FBE0F901F9018951F92BD
:100B90000F920FB60F9211242F933F934F935F93B1
:100BA0006F937F938F939F93AF93BF93EF93FF9335
:100BB0008091B900887F803609F49CC068F588323E
:100BC00009F45BC090F4803109F454C038F48823F0
:100BD00009F4F6C0883009F44DC0F6C0883109F434
:100BE0004CC0803209F45DC0EFC0803409F468C0A5
:100BF00048F4803309F455C0883309F0E5C0809388
:100C00002603D8C0803509F44FC0883509F45DC08B
:100C1000883409F0D9C0D6C0883909F4C7C0A8F40F
:100C2000883709F467C038F4883609F463C0803720
:100C300009F460C0C9C0883809F4B8C0803909F423
:100C40005FC0803809F0C0C05BC0803B09F486C03B
:100C500038F4803A09F466C0883A09F47FC0B4C019
:100C6000803C09F4A7C0883C09F4A4C0883B09F47F
:100C70008AC0AAC08091030310C09091250380917F
:100C80002403981770F5E091250381E08E0F80937F
:100C90002503F0E0EC5FFC4F80818093BB0085EC86
:100CA00086C0809326038EC0E091250381E08E0FDD
:100CB000809325038091BB00F0E0EC5FFC4F8083C4
:100CC00090912503809124036EC0E091250381E07B
:100CD0008E0F809325038091BB00F0E0EC5FFC4F0A
:100CE00080838091270381116DC081E0809302038E
:100CF00084EA61C083E0809328031092DA02CFCFA8
:100D00008091DA02803208F051C0E091DA0281E08D
:100D10008E0F8093DA028091BB00F0E0E654FD4F25
:100D20008083BDCF85EC8093BC0010922803809116
:100D3000DA02803230F4E091DA02F0E0E654FD4F5E
:100D400010826091DA0270E0E091B802F091B9028D
:100D50008AEB92E009951092DA0236C084E0809323
:100D600028031092B7021092B602E091B402F091FB
:100D7000B50209958091B602811105C081E080938A
:100D8000B60210929402E091B70281E08E0F809338
:100D9000B702F0E0EC56FD4F80818093BB0090914C
:100DA000B7028091B602981708F479CF85E880934E
:100DB000BC000AC085EC8093BC001092280304C0DC
:100DC000109226030E940C02FF91EF91BF91AF9108
:100DD0009F918F917F916F915F914F913F912F9153
:100DE0000F900FBE0F901F901895CF92DF92EF9249
:100DF000FF920F931F93CF93DF937C016C0187E0E9
:100E0000C80ED11CC0E0D0E0062F10E0B8010C2EB7
:100E100002C0759567950A94E2F76170F6018191B9
:100E20006F010E94C1042196C430D10579F7C70132
:100E3000DF91CF911F910F91FF90EF90DF90CF90B6
:100E40000C94F104CF92DF92EF92FF920F931F93D5
:100E5000CF93DF93EC01F62E642F8C810E94C104A6
:100E60008D818F3F19F060E00E94C1048F850F2DA6
:100E700010E084FF25C06E0187E0C80ED11CE12C74
:100E8000F12CB8010E2C02C0759567950A94E2F713
:100E90006170F60181916F010E94C104FFEFEF1AAA
:100EA000FF0A88E0E816F10461F7CE01DF91CF91E7
:100EB0001F910F91FF90EF90DF90CF900C94F10471
:100EC000B80184E0759567958A95E1F7CE010E9497
:100ED000F5066F2DCE01DF91CF911F910F91FF90FD
:100EE000EF90DF90CF900C94F50641E00E9422072E
:100EF00081E090E0089540E00C942207CF92DF92C9
:100F0000FF920F931F93CF93DF9300D000D0CDB704
:100F1000DEB78E010F5F1F4F6C01C01AD10A84E04B
:100F2000F82EF00EC601800F911F0E94AD24F8012B
:100F300081938F01FE12F6CF69817A818B819C812A
:100F40000F900F900F900F90DF91CF911F910F9105
:100F5000FF90DF90CF900895CF92DF92EF92FF92B3
:100F60008AE090E00E947E07609390027093910265
:100F700080939202909393026A3F710581059105D7
:100F800081F040EB5AE262E070E080E090E00E9485
:100F9000CB024AEF50E060E070E08AE090E00E940F
:100FA000CB0280915A02813091F580E090E00E945E
:100FB0007E076B017C0120915B0230915C024091C5
:100FC0005D0250915E0260914E0270914F028091DD
:100FD0005002909151020E941425AB01BC014C0DAE
:100FE0005D1D6E1D7F1D4093560250935702609306
:100FF00058027093590280E090E00E94CB024AEFC1
:1010000050E060E070E08AE090E00E94CB0280E077
:1010100090E00E947E07609356027093570280937F
:10102000580290935902FF90EF90DF90CF9008956F
:101030001F920F920FB60F9211242F933F934F934D
:101040005F936F937F938F939F93AF93BF93CF9350
:10105000DF93EF93FF93809188040E94BE01EC011F
:10106000809187040E94BE01CC0FDD1F8C2BE09184
:101070008604EF7094E0E99FF0011124E80FF11D60
:10108000E65FFE4F8081809386048073803161F437
:1010900080915B0290915C02A0915D02B0915E0232
:1010A0000196A11DB11D0DC0803299F480915B02A3
:1010B00090915C02A0915D02B0915E020197A1093E
:1010C000B10980935B0290935C02A0935D02B093A0
:1010D0005E02FF91EF91DF91CF91BF91AF919F9110
:1010E0008F917F916F915F914F913F912F910F90D1
:1010F0000FBE0F901F9018952F923F924F925F92C4
:101100006F927F928F929F92AF92BF92CF92DF9217
:10111000EF92FF920F931F93CF93DF93CDB7DEB77C
:101120006A970FB6F894DEBF0FBECDBF322E232EC6
:101130004D875E873B012C01A982B98ACA8ADB8A66
:10114000EC8AFD8A0E8B1F8B988A8F86211500EA08
:1011500030070CEA400709EB500703E06007710510
:101160008105910511F008F046C02F3F10EE3107C0
:1011700015EF410715E051076105710581059105DE
:1011800061F058F02F3F354D41415E476340710596
:101190008105910509F0D8F50BC0312CB1EE2B2E4D
:1011A000F5EFFD8705E00E87612C712C412C512C49
:1011B000298139894A895B896C897D898E899F89D2
:1011C000A0E00E94F02609F0AEC0A32CB22CCD8482
:1011D000DE847301820120E034E04BE654EF64E1E9
:1011E00070E080E090E00E94312629873A874B87A3
:1011F0005C87912C24C0312CF0EA2F2E1CEA1D872D
:1012000029EB2E87A3E06A2E712C412C512C2981C9
:1012100039894A895B896C897D898E899F89A0E09B
:101220000E94F02609F025C19924939414E0E12E40
:10123000F12C00E010E0E986FA860B871C87E98430
:10124000FA840B851C85A801970160E070E0CB0152
:10125000A32CB22CCD84DE847301820129833A83CE
:101260004B835C836D837E838F83988760E070E01F
:1012700080E090E00E946B252983398B4A8B5B8B41
:101280006C8B7D8B8E8B9F8BFF24F3949F1409F4C2
:10129000F3C010E0812C912C54018394C12CD12CEB
:1012A000760101C011E007E0CC0CDD1CEE1CFF1C38
:1012B0000A95D1F7C701B601A50194010E94242522
:1012C00089859A85AB85BC8567E0880F991FAA1F21
:1012D000BB1F6A95D1F79250A109B109820F931FE4
:1012E000A41FB51FEF85F88980839183A283B38300
:1012F000C501B4010E941425C61AD70AE80AF90AE2
:10130000C482D582E682F78280869186A286B386E1
:101310001111E5C0298139894A895B896C897D89E8
:101320008E899F89E2C01A8EA32CB22CCD84DE84D4
:1013300073018201298139894A895B896C897D8998
:101340008E899F890E94312629873A874B875C873F
:1013500089859A85AB85BC850697A105B10520F4E2
:10136000F6E0AF2EB12C0FC0E984FA840B851C8502
:1013700029E0E21627E0F20601051105D0F078E039
:10138000A72EE7E0BE2EC12CD12CE12CF12C00E0E1
:1013900010E0298139894A895B896C897D898E8928
:1013A0009F890E943126322E232E4D875E873B0176
:1013B0002C01A32CB22CCD84DE84730182012981FF
:1013C00039894A895B896C897D898E899F890E94C8
:1013D0002F264901B42FA52FF62FE72F888F998F3D
:1013E00005E00E949E265401CB2EDA2EEF2EFE2E13
:1013F000088D198D0E94DE2605E00E949E26088D2C
:101400000E94D52605E00E949E26088D0E94DE26B9
:10141000288F398F4A01B62FA72FF82FE92F6B2F6E
:101420007A2F8F2F9E2F05E00E949E2659016A0178
:101430007B018C01288D398DA4016B2F7A2F8F2F82
:101440009E2F0E94D526A32CB22CCD84DE8473015E
:1014500082010E943126C22ED32EE42EF52EC11415
:10146000D104E104F104F9F4812C912C540183940A
:1014700020C081E08A8F58CFAF85B8891D921D9218
:101480001D921C921397FD011482158216821782F9
:10149000C12CD12C7601C3941896CD92DD92ED9299
:1014A000FC921B9722C088248A94982C8FE0A82E47
:1014B000B12CFA8DF13009F0F5CEEF85F889108264
:1014C000118212821382148215821682178281E0A1
:1014D00090E0A0E0B0E080879187A287B387232DBA
:1014E000322D4D855E85B301C2016A960FB6F89420
:1014F000DEBF0FBECDBFDF91CF911F910F91FF9047
:10150000EF90DF90CF90BF90AF909F908F907F90A3
:101510006F905F904F903F902F900895DF92EF92E1
:10152000FF920F931F93CF93DF93FC01E080F18034
:1015300002811381D481C581B681D7809701A8012A
:101540006D2F7C2F8B2F9D2D35534C4051096109F8
:101550007109810991092F3F34434C4051056105C0
:1015600071058105910509F098F49701A8016D2F87
:101570007C2F8B2F9D2D07E00E949E262083318398
:1015800042835383648375838683978387E0FDC09A
:101590009701A8016D2F7C2F8B2F9D2D3A56484126
:1015A000510961097109810991092F3F3946484163
:1015B0005105610571058105910509F098F49701C0
:1015C000A8016D2F7C2F8B2F9D2D06E00E949E265B
:1015D0002083318342835383648375838683978317
:1015E00086E0D3C09701A8016D2F7C2F8B2F9D2DF6
:1015F000345D4043510961097109810991092F3F07
:10160000334D40435105610571058105910509F090
:1016100098F49701A8016D2F7C2F8B2F9D2D05E04D
:101620000E949E2620833183428353836483758383
:101630008683978385E0A9C09701A8016D2F7C2F31
:101640008B2F9D2D385A4146510961097109810935
:1016500091092F3F374A41465105610571058105C2
:10166000910509F098F49701A8016D2F7C2F8B2F1D
:101670009D2D04E00E949E26208331834283538364
:10168000648375838683978384E07FC09701A80174
:101690006D2F7C2F8B2F9D2D3055434C51096109A7
:1016A0007109810991092F3F3F44434C5105610560
:1016B00071058105910509F098F49701A8016D2F36
:1016C0007C2F8B2F9D2D03E00E949E26208331834B
:1016D00042835383648375838683978383E055C0F5
:1016E0009701A8016D2F7C2F8B2F9D2D305A4648D6
:1016F000514061097109810991092F3F3F494648CD
:101700005140610571058105910509F098F4970133
:10171000A8016D2F7C2F8B2F9D2D02E00E949E260D
:1017200020833183428353836483758386839783C5
:1017300082E02BC09701A8016D2F7C2F8B2F9D2D50
:1017400030544D40534061097109810991092F3F7F
:101750003F434D405340610571058105910509F0F6
:1017600098F49701A8016D2F7C2F8B2F9D2D01E000
:101770000E949E2620833183428353836483758332
:101780008683978381E001C080E0DF91CF911F9134
:101790000F91FF90EF90DF900895CF93DF9391E04A
:1017A0009093290390E690934B0310922A03109292
:1017B0004C03682F8AEE93E00E949A0281E00E9417
:1017C0007612809128038111FCCF91E09093280339
:1017D000109227038FEF8093260310922503109217
:1017E00024039093030390910303906C909303035D
:1017F00080910203813061F410920203809103030F
:101800008093BB008091BC0083FDF8CF85EC01C0C4
:1018100085EE8093BC00809128038130E1F38091B4
:101820002503811103C0C091250301C0C1E0A4E0DC
:10183000B3E022EE32E0F9018E2F821B8C1718F4F0
:101840008D918193F9CF1092E102C093E0028091D3
:10185000E102C81731F08AEE93E00E944E02D82FC1
:10186000F6CF8D2FDF91CF9108952F923F924F9217
:101870005F926F927F928F929F92AF92BF92CF9220
:10188000DF92EF92FF920F931F93CF93DF93CDB729
:10189000DEB72E970FB6F894DEBF0FBECDBF982EE1
:1018A000792E49875A876B877C876BA05C2C2D2CFF
:1018B0003E2D402E312EC984DA84EB84FC8484E1F1
:1018C00090E02E873D870E94FC268C01FC01D0828F
:1018D000C182892D880F880F880F845D0E94CD0BEF
:1018E0008C7F3D85932F9370892BF801828323820F
:1018F0005482D701C6016CE0B695A7959795879558
:101900006A95D1F7982F907F2E85822F8F70C82EE1
:10191000C90EC58236824782E92CF72CF8E0EF1613
:10192000F104B8F4F701EC5CFF4FB8010C946525A5
:101930008AE20DC082E30BC08AE309C082E407C0DB
:101940008AE405C082E503C08AE501C08BE50E94F8
:10195000D31280E1980E892D0E94CD0B91E0682F63
:10196000A91202C0606401C06F7B892D0E94F2142D
:10197000E1E0EE16F10451F0F2E0EF16F10449F067
:10198000E114F10449F4A092BA0412C0A092BB047D
:1019900012C0A092BC0412C088E0E816F104B0F4B2
:1019A000F701E45CFF4F0C94652554E4B52E0EC09E
:1019B0004CE2B42E0BC034E3B32E08C02CE3B22E9D
:1019C00005C09CE4B92E02C084E5B82E8B2D0E9480
:1019D000CD0B837861108C6090E1899E40011124C9
:1019E000682F68298B2D0E94F214C8012E960FB61D
:1019F000F894DEBF0FBECDBFDF91CF911F910F9145
:101A0000FF90EF90DF90CF90BF90AF909F908F901E
:101A10007F906F905F904F903F902F900C94912704
:101A20000F931F93CF938B01C0E1C80F8C2F0E949F
:101A3000CD0B0115110511F48F7D04C00130110586
:101A400009F48062682F8C2FCF911F910F910C9415
:101A5000F2142F923F924F925F926F927F928F92E9
:101A60009F92AF92BF92CF92DF92EF92FF920F932D
:101A70001F93CF93DF93CDB7DEB7AA970FB6F89435
:101A8000DEBF0FBECDBF622E298F732E3A8F4B8FD4
:101A90005C8F6D8F7E8F8F8F98A319A708A79301F6
:101AA0002F3F34434C405105610571058105910577
:101AB00009F050F4198E85E38A8F8CE08B8F1C8E91
:101AC0001D8E1E8E1F8E18A2298D3A8D4B8D5C8D1A
:101AD0006D8D7E8D8F8D98A12115304A4C4A594BC2
:101AE000634071058105910569F060F0198E80EA07
:101AF0008A8F8CEA8B8F89EB8C8F83E08D8F1E8E83
:101B00001F8E18A2CE0149960E948E0A8AA7798C50
:101B1000BA8DAB8DFC8DED8D6E8C5F8C48A0272D22
:101B20003B2F4A2F5F2F6E2F762D852D942D2F3F23
:101B300005ED300701E140070EE7500703E06007BD
:101B400071058105910511F008F081C09E01235FA8
:101B50003F4F4901A12CE8E5BE2EF7E4CF2EA8EFB8
:101B6000DA2E1DE0E12EF12C00E010E0272D3B2FB6
:101B70000E947C0888A599A58130910559F1823091
:101B8000910509F440C0892B09F05DC3898D8093CC
:101B9000A2048A8D8093A3048B8D8093A4048C8DE2
:101BA0008093A5048D8D8093A6048E8D8093A704C9
:101BB0008F8D8093A80488A18093A90480E019A246
:101BC000212C58E5352E67E4462E98EF9CA3EDE0D6
:101BD000EDA344C3898D8093AA048A8D8093AB04BE
:101BE0008B8D8093AC048C8D8093AD048D8D809310
:101BF000AE048E8D8093AF048F8D8093B00488A146
:101C00008093B10420C3898D8093B2048A8D809320
:101C1000B3048B8D8093B4048C8D8093B5048D8D2B
:101C20008093B6048E8D8093B7048F8D8093B80413
:101C300088A18093B90480E019A2212C38E5332EC5
:101C400047E4442E18EF1CA32DE02DA307C3CE01BB
:101C50000D964C01A12CB12CC12CD12CE12CF12CD6
:101C600000E010E0272D3B2F4A2F5F2F6E2F762D9F
:101C7000852D942D0E947C08E8A5F9A5E130F10599
:101C800009F450C0E230F10509F492C1EF2B09F0DC
:101C90000BC3298D3A8D4B8D5C8D6D8D7E8D00E053
:101CA00010E08F8D98A10E947C081901442E5CA33E
:101CB0006DA3772E582E692E60E070E080E090E0F2
:101CC0000E94100D2092920430929304409294044A
:101CD0001CA1109395042DA1209396047092970453
:101CE0005092980460929904898D8093A2048A8D01
:101CF0008093A3048B8D8093A4048C8D8093A50482
:101D00008D8D8093A6048E8D8093A7048F8D8093F4
:101D1000A80488A18093A90481E031E039A31BA223
:101D20001AA29FC21091C204B98DAA8DFB8DEC8DB1
:101D30000D8D09A30E8D0AA30F8D0EA308A10FA36D
:101D4000123009F073C02B2F3A2F4F2F5E2F69A14D
:101D50007AA18EA1902F30584A41564061097109ED
:101D6000810991092F37304E424758496240710529
:101D70008105910569F160F1A090B204B090B304BF
:101D8000C090B404D090B504E090B604F090B704CD
:101D90000091B8041091B9042B2F3A2F4F2F5E2FCA
:101DA00069A17AA18EA19FA10E94E72689F01092D5
:101DB000AA041092AB041092AC041092AD041092DD
:101DC000AE041092AF041092B0041092B1046CC231
:101DD00020909A0430909B0440909C0420919D0494
:101DE0002CA330919E043DA370909F045090A004BA
:101DF0006090A104CE010D964C015101C42CD22E4D
:101E0000E32EF72C052D162D2B2F3A2F4F2F5E2F5B
:101E100069A17AA18EA19FA10E947C0861E070E077
:101E200081E090E00E94100D19A235C020939A0421
:101E300030939B0440939C0450939D0460939E04B4
:101E400070939F048093A0049093A1048E01035F7C
:101E50001F4F4801A12CB12CC12CD12CE12CF12C0D
:101E600000E010E02B2F3A2F4F2F5E2F69A17AA1AF
:101E70008EA19FA10E947C081901442E5CA36DA332
:101E8000772E582E692E61E070E081E090E00E948C
:101E9000100D11E019A3298D3A8D4B8D5C8D6D8D40
:101EA0007E8D8F8D98A130584A4156406109710945
:101EB000810991092F37304E4247584962407105D8
:101EC0008105910509F008F457C081E08093C204B0
:101ED0002091B2043091B3044091B4045091B50400
:101EE0006091B6047091B7048091B8049091B904E0
:101EF000A0E00E94F02609F442C082EB94E00E9428
:101F00008E0A8AA7A0909A04B0909B04C0909C046B
:101F1000D0909D04E0909E04F0909F040091A00456
:101F20001091A1042091B2043091B3044091B40403
:101F30005091B5046091B6047091B704CE0101963A
:101F40004C018091B8049091B9040E947C081F92C2
:101F50008AA4A12CC980DA80EB80FC800D811E81CF
:101F60002F81388549855A856B857C8582E090E094
:101F70000E94350C0F9003C088E08093C204898DC5
:101F80008093AA048A8D8093AB048B8D8093AC04DC
:101F90008C8D8093AD048D8D8093AE048E8D809357
:101FA000AF048F8D8093B00488A18093B10445C1A4
:101FB0007090C204B98DAA8DFB8DEC8D0D8D09A397
:101FC0001E8D1AA30F8D0EA318A11FA301E070127E
:101FD00073C02B2F3A2F4F2F5E2F69A17AA18EA1AC
:101FE000912F30584A415640610971098109910980
:101FF0002F37304E4247584962407105810591059F
:1020000069F160F1A090B204B090B304C090B40440
:10201000D090B504E090B604F090B7040091B804F5
:102020001091B9042B2F3A2F4F2F5E2F69A17AA15F
:102030008EA19FA10E94E72689F01092B20410920F
:10204000B3041092B4041092B5041092B604109226
:10205000B7041092B8041092B9042AC120909A04CF
:1020600030909B0440909C0420919D042CA33091BF
:102070009E043DA370909F045090A0046090A10422
:10208000CE010D964C015101C42CD22EE32EF72C1B
:10209000052D162D2B2F3A2F4F2F5E2F69A17AA1D8
:1020A0008EA19FA10E947C0861E070E082E090E038
:1020B0000E94100D19A235C020939A0430939B04FE
:1020C00040939C0450939D0460939E0470939F04DE
:1020D0008093A0049093A1048E01035F1F4F4801D9
:1020E000A12CB12CC12CD12CE12CF12C00E010E062
:1020F0002B2F3A2F4F2F5E2F69A17AA18EA19FA17E
:102100000E947C081901442E5CA36DA3772E582EE3
:10211000692E61E070E082E090E00E94100D11E015
:1021200019A3298D3A8D4B8D5C8D6D8D7E8D8F8D94
:1021300098A130584A4156406109710981099109B5
:102140002F37304E4247584962407105810591054D
:1021500009F008F457C082E08093C2042091AA04D9
:102160003091AB044091AC045091AD046091AE0449
:102170007091AF048091B0049091B104A0E00E94EE
:10218000F02609F442C08AEA94E00E948E0A8AA7E7
:10219000A0909A04B0909B04C0909C04D0909D04A1
:1021A000E0909E04F0909F040091A0041091A1047F
:1021B0002091AA043091AB044091AC045091AD043D
:1021C0006091AE047091AF04CE0101964C018091F4
:1021D000B0049091B1040E947C081F928AA4A12CA3
:1021E000C980DA80EB80FC800D811E812F813885CB
:1021F00049855A856B857C8581E090E00E94350C8D
:102200000F9003C088E08093C204898D8093B2044C
:102210008A8D8093B3048B8D8093B4048C8D8093CE
:10222000B5048D8D8093B6048E8D8093B7048F8D09
:102230008093B80488A18093B90481E0E1E0F0E0E4
:10224000FBA3EAA30EC080E019A2212C98E5392E49
:1022500027E4422EF8EFFCA30DE00DA3712C512CC6
:10226000612C8F938AA4A82ECD84DE84EF84F88815
:1022700009891A892B893C894D895E896F89788DF6
:1022800088A599A50E94350C0F9019A1113079F4F9
:102290000AA11BA19101442D5CA16DA1772D852D73
:1022A000962D0E94071303C07724739401C0712CEC
:1022B000872DAA960FB6F894DEBF0FBECDBFDF9173
:1022C000CF911F910F91FF90EF90DF90CF90BF9033
:1022D000AF909F908F907F906F905F904F903F90C6
:1022E0002F90089580E480937C0080917A00806430
:1022F00080937A0080917A0086FDFCCF80917800EF
:102300002091790090E0922B08958F929F92AF9246
:10231000BF920F931F93CF93DF93CDB7DEB7A197F3
:102320000FB6F894DEBF0FBECDBF19A2423008F43D
:102330004AE08E010F5D1F4F842E912CA12CB12CF1
:10234000A50194010E942425E62FB901CA0101507C
:102350001109EA3014F4E05D01C0E95CD801EC93A6
:10236000232B242B252B61F7B80186EF93E00E94E5
:102370005204A1960FB6F894DEBF0FBECDBFDF9119
:10238000CF911F910F91BF90AF909F908F90089524
:10239000E091F603F091F7030190F081E02D682FB2
:1023A00086EF93E00994EF92FF920F931F93CF93E0
:1023B000DF93EC01623018F08F8588608F876B8B1C
:1023C0001C8A80E48D8B80E18E8B80E58F8B61E0B1
:1023D0008C810E9407058D818F3F19F061E00E947A
:1023E000070561E08E810E9407057E0187E0E80E07
:1023F000F11C00E010E08F8584FD03C084E090E0D4
:1024000002C088E090E0081719074CF461E0F7017A
:1024100081917F010E9407050F5F1F4FECCF8BE377
:102420009DE00197F1F760E08C810E94C10460E0BB
:102430008E810E94C1048D818F3F19F060E00E945F
:10244000C1046F8564FD1DC063E0CE010E94F506E6
:102450000BE416E4C8010197F1F763E0CE010E9496
:10246000F506C8010197F1F763E0CE010E94F50679
:1024700083E592E00197F1F762E0CE010E94F50654
:1024800016C06062CE010E947B078BE496E4019740
:10249000F1F76F856062CE010E947B0783E592E0D1
:1024A0000197F1F76F856062CE010E947B076F850F
:1024B0006062CE010E947B0784E0888B6CE0CE01D5
:1024C0000E947B0761E0CE010E947B078BE39FE1C6
:1024D0000197F1F782E0898B66E0CE01DF91CF9121
:1024E0001F910F91FF90EF900C947B07382F209154
:1024F0004C0390914B03213208F049C0809128038E
:102500008111FCCF42E040932803309327033FEF33
:10251000309326031092250320932403ABE2B3E00B
:1025200044E053E0FA013E2F341B321718F43D917A
:102530003193F9CF1092030320910303990F922B4B
:102540009093030390910203913061F4109202037F
:10255000909103039093BB009091BC0093FDF8CF42
:1025600095EC01C095EE9093BC00909128039230B9
:10257000E1F3909126039F3F79F08091260380320A
:1025800041F080912603803331F084E005C081E082
:1025900003C082E001C083E010922A0310924C0332
:1025A000109229030895EF92FF920F931F93CF93F8
:1025B000DF931F92CDB7DEB7162F91E090932903DA
:1025C00090E690934B0310922A0310924C03682FCD
:1025D0008AEE93E079830E949A02E12E7981F72EA8
:1025E0008701085F1F4FF70161917F018AEE93E039
:1025F0000E949A02E016F106B1F781E00F90DF9198
:10260000CF911F910F91FF90EF900C9476122F9223
:102610003F924F925F926F927F928F929F92AF9272
:10262000BF92CF92DF92EF92FF920F931F93CF93BF
:10263000DF93CDB7DEB763970FB6F894DEBF0FBE5A
:10264000CDBF322E3A874B875C876D87272E2C01B2
:102650001F870E876091C3047091C4048091C504E4
:102660009091C60424E630E040E050E00E94D3257B
:102670002A8B3B8B4D835E83762E672E888B998BBE
:102680008091BD049091BE04A091BF04B091C0049C
:102690006C017D01FF0CCC08DC2C76019C01AD01A6
:1026A0006C2D7C2D8C2D9C2D0FE10E949E26A12C43
:1026B000EAECBE2EFAE9CF2EABE3DA2EE12CF12CB8
:1026C00000E010E00E940026AA88BB88CD80DE8052
:1026D000E72CF62C088919890E946B250FE10E94CE
:1026E000B92649015A01D501C401BB0F880B982FA7
:1026F000DC0189839A83AB83BC839401A501698142
:10270000762F862F962FAA88BB88CD80DE80E72C77
:10271000F62C08890E94D52639014A01698B788BED
:1027200089839D83232D3A854B855C856D85722D2C
:10273000C2012F3FA7E53A07A7E44A07A8EF5A07C7
:10274000ADE06A07710581059105A9F0A0F021159A
:1027500034404B46544F6441710581059105B9F0F1
:10276000B0F0312CA4E0AA87BBE6BB87E4EFEC878E
:10277000F4E1FD8709C0312CE8E5EA87F7E4FB873F
:1027800088EF8C879DE09D87212C412C512C530193
:102790006401E988F88809811D81232D3A854B85DC
:1027A0005C856D85722DC2010E9431262E833F8388
:1027B000488759878E819F81A885B9850F97A10584
:1027C000B10558F49301A401B701C80104E00E94C7
:1027D0009E2609810E94DE2628C08E819F81A885C1
:1027E000B9858B359105A105B10530F19301A4019F
:1027F0006989788989819D8102E00E949E26530122
:102800006401E988F88809811D810E94DE2659014A
:102810006A017B01E82F192F04E00E949E260E2FEB
:102820000E94DE2601E00E949E26322E3A874B87C8
:102830005C876D87272E2C0153016401E988F88895
:1028400009811D81232D3A854B855C856D85722D0F
:10285000C2010E942F262901B42FA52FF62FE72FA2
:10286000382E292E05E00E949E265201CB2EDA2E0C
:10287000EF2EFE2E032D122D0E94DE2605E00E9473
:102880009E26032D0E94D52605E00E949E26032D3C
:102890000E94DE2619012A01B62FA72FF82FE92F53
:1028A00005E00E949E2659016A017B018C0191017D
:1028B000A2016B2F7A2F8F2F9E2F0E94D5265301B6
:1028C0006401E988F88809811D810E943126690127
:1028D0007A01C114D104E104F10429F4812C912C72
:1028E0005401839406C088248A94982C3FE0A32E38
:1028F000B12C87E0CC0CDD1CEE1CFF1C8A95D1F7B7
:10290000C701B601A50194010E9424254E805F8075
:102910006884798497E0440C551C661C771C9A9552
:10292000D1F792E0591A61087108420E531E641ED5
:10293000751EC501B4010E941425C61AD70AE80AFB
:10294000F90A84E190E00E94FC268C01DC019C9253
:1029500011968C921197862D837012968C931297F4
:1029600013965C92139714964C92D501C4012CE0F7
:10297000B695A795979587952A95D1F7982F907F2B
:102980008E2D8F70882E890EF8018582D682C7829F
:102990008E859F85892B19F4B8018AE106C0AE8522
:1029A000BF85119721F4B80182E20E94D312C801B9
:1029B00063960FB6F894DEBF0FBECDBFDF91CF9107
:1029C0001F910F91FF90EF90DF90CF90BF90AF904D
:1029D0009F908F907F906F905F904F903F902F903F
:1029E0000C949127CF93C62F91E09093290390E602
:1029F00090934B0310922A0310924C03682F8AEE97
:102A000093E00E949A026C2F8AEE93E00E949A0251
:102A100081E0CF910C947612643008F063E09091DD
:102A20000904691710F06FEF690FE62FF0E0EA5024
:102A3000FC4F9489682F690F606886EF93E00C94CF
:102A40007B07FC0180914E0490914F04892B21F467
:102A500021E0309749F413C080914A0490914B04CF
:102A6000309731F421E0FC018081882341F006C0D9
:102A7000BF010E94012921E0892B09F020E0822F6B
:102A80000895CF93DF9300D0CDB7DEB789831A8244
:102A900041E050E0BE016F5F7F4F80E894E00E940C
:102AA00063030F900F90DF91CF910895CF93DF9341
:102AB000CDB7DEB7E2970FB6F894DEBF0FBECDBF3D
:102AC000789484B5826084BD84B5816084BD85B509
:102AD000826085BD85B5816085BD80916E00816015
:102AE00080936E00109281008091810082608093BB
:102AF00081008091810081608093810080918000BD
:102B00008160809380008091B10084608093B100E7
:102B10008091B00081608093B00080917A008460E1
:102B200080937A0080917A00826080937A0080910D
:102B30007A00816080937A0080917A008068809327
:102B40007A001092C100E0915D03F0915E0382E093
:102B50008083E0915D03F0915E031082E091590360
:102B6000F0915A031082E0915B03F0915C0380E1E5
:102B7000808310926503E0916103F091620386E027
:102B80008083E0915F03F0916003808180618083A6
:102B9000E0915F03F0916003808188608083E09121
:102BA0005F03F0916003808180688083E0915F0320
:102BB000F091600380818F7D808362E086EF93E0F7
:102BC0000E94D31160E470E080E894E00E943C032E
:102BD00060E08EE00E94070561E08FE00E9407053B
:102BE00061E080E10E94070561E081E10E94070544
:102BF00061E084E10E94070561E085E10E9407052C
:102C000061E08AE00E94070561E08BE00E94070511
:102C100061E08CE00E94070561E08DE00E940705FD
:102C200061E08FE00E94070561E080E10E940705F6
:102C300061E081E10E94070561E084E10E940705EF
:102C400061E085E10E94070560E08FE00E94C10419
:102C500060E080E10E94C10460E081E10E94C10463
:102C600061E084E10E94C10461E085E10E94C10449
:102C70008091680084608093680080916D008C6012
:102C800080936D00789480E090E00E947E076093CE
:102C900056027093570280935802909359026093A2
:102CA000BD047093BE048093BF049093C00410923F
:102CB000E1021092E00210922A0310924C0310924B
:102CC000280381E0809327031092020361E082E1F0
:102CD0000E94C10461E083E10E94C1048091B900B7
:102CE0008E7F8093B9008091B9008D7F8093B90069
:102CF00088E48093B80085E48093BC0062E987EBA8
:102D00000E94F21460E880E10E94F21460E881E120
:102D10000E94F21460E882E10E94F2146CE080E10B
:102D20000E94F2146CE081E10E94F2146CE082E1F6
:102D30000E94F21460E281EB0E94F21460E881EBE1
:102D40000E94F21400E010E020E038E547E458EF7C
:102D50006DE070E080E090E00E9407138091000138
:102D600090910101A0910201B0910301BC01CD013C
:102D700032E0660F771F881F991F3A95D1F724E636
:102D800030E040E050E00E94C4250E94290D80E11F
:102D90000E94CD0B682F636080E10E94F21440E432
:102DA000842E42E4942E4FE0A42EB12C52E3452E03
:102DB000512C612C712C0E94AC0720915B02309148
:102DC0005C0240915D0250915E0221153105410582
:102DD000510509F4B0C060914E0270914F0280918C
:102DE0005002909151020E941425009160021091AE
:102DF00061022091620230916302600F711F821F95
:102E0000931F6093600270936102809362029093BB
:102E100063021AA619A61CA61BA61EA61DA62AE0BA
:102E2000AE014F5F5F4F0E943D24BE016F5F7F4F39
:102E3000CE0189960E94C4038DA59EA50B9778F5B7
:102E40001CA21BA21EA21DA218A61FA24AE0BE0120
:102E50006F5F7F4F80E090E00E943224BE016F5F81
:102E60007F4FCE0183960E94C4034DA55EA569A540
:102E70007AA5CE0183960E946303811104C0CE011E
:102E800083960E949103BE016D5D7F4FCE018996AE
:102E90000E94DB03CE0183960E94F203CDCF6EE445
:102EA00071E0CE0101960E94F7034DA55EA569A5CC
:102EB0007AA5CE0101960E946303811104C0CE0160
:102EC00001960E94910341E050E06FEA71E0CE016B
:102ED00001960E946303882311F40C945A22BE01C8
:102EE0006F5F7F4FCE0189960E94DB03CE01019672
:102EF0000E94F20380915A02813019F40E94AC07BB
:102F00000EC04DA55EA569A57AA58DE493E00E944B
:102F10009E0063E270E080E090E00E944305109222
:102F20005B0210925C0210925D0210925E02CE0172
:102F300089960E94F20361E571E08DE493E00E94BE
:102F400067048DE493E00E94690168E270E080E02C
:102F500090E00E9443058DE493E00E94EB00892BF2
:102F6000D9F580915F02811109C061E086EF93E09D
:102F70000E947B078BE39FE10197F1F760E080E01F
:102F80000E940C1565E571E086EF93E00E946704EE
:102F900064EF71E080E090E00E94430561E080E032
:102FA0000E940C1566E671E086EF93E00E946704CC
:102FB00068EE73E080E090E00E94430561E080E00D
:102FC0000E940C1567E771E086EF93E00E946704AA
:102FD00081E080935F02AFCF8DE493E00E94EB002D
:102FE0001816190644F58DE493E00E94C9008093F9
:102FF0007202893439F0809171028823E1F01092D5
:10300000710219C089E40E94411501E08DE493E04A
:103010000E94EB001816190674F78DE493E00E94E5
:10302000C900182F809372020E9441151B3371F75B
:1030300000937102EBCF1CA21BA21EA21DA218A618
:103040001FA260E874E0CE0183960E94DB032DE0AE
:1030500030E042E050E0BE016D5D7F4FCE01019651
:103060000E940C04BE016F5F7F4F82E694E00E94D5
:103070000303CE0101960E94F20382E694E00E94CF
:10308000F802609300017093010180930201909314
:103090000301809184028130A1F480918A02813001
:1030A00081F480916D0290916E02A0916F02B091B7
:1030B00070028093000190930101A0930201B093EC
:1030C0000301C0900001D0900101E0900201F09056
:1030D0000301C0926002D0926102E0926202F0921B
:1030E00063022EE130E04DE150E0BE016D5D7F4FA7
:1030F000CE0101960E940C04BE016F5F7F4F8CE5EC
:1031000094E00E940303CE0101960E94F2038CE535
:1031100094E00E94F8026093830221E230E040E2F2
:1031200050E0BE016D5D7F4FCE0101960E940C0400
:10313000BE016F5F7F4F86E294E00E940303CE01E1
:1031400001960E94F20386E294E00E94F8026093E6
:10315000840228E130E047E150E0BE016D5D7F4F21
:10316000CE0101960E940C04BE016F5F7F4F84E781
:1031700094E00E940303CE0101960E94F20384E7CB
:1031800094E00E94F8026093820229E130E048E175
:1031900050E0BE016D5D7F4FCE0101960E940C0490
:1031A000BE016F5F7F4F8EE694E00E940303CE0165
:1031B00001960E94F2038EE694E00E94F80260936A
:1031C000810221E130E04DE050E0BE016D5D7F4FB6
:1031D000CE0101960E940C04BE016F5F7F4F86E511
:1031E00094E00E940303CE0101960E94F20386E55B
:1031F00094E00E94F802709365026093640222E1F9
:1032000030E041E150E0BE016D5D7F4FCE0101969F
:103210000E940C04BE016F5F7F4F8AE494E00E941D
:103220000303CE0101960E94F20327E130E042E160
:1032300050E0BE016D5D7F4FCE0101960E940C04EF
:10324000BE016F5F7F4F80E594E00E940303CE01D3
:1032500001960E94F20380E594E00E94F8026093D8
:103260007D0270937E0280937F02909380022DE115
:1032700030E04CE150E0BE016D5D7F4FCE01019624
:103280000E940C04BE016F5F7F4F8AE794E00E94AA
:103290000303CE0101960E94F2038AE794E00E94A4
:1032A000F80260938A0267E871E080E894E00E9487
:1032B000C403CE0183960E94F20380918C02909108
:1032C0008D02A0918E02B0918F02C816D906EA062F
:1032D000FB0609F49BC0D701C60180549244AF405D
:1032E000B10980389448AE41B10518F415B880EAA8
:1032F00086C0D701C601805C964CAD42B1098038CA
:103300009448AE41B10520F484E085B980E577C0EA
:10331000D701C60180549B44AC44B109803C964C13
:10332000AD42B10520F488E085B988E268C0D701D4
:10333000C6019251AA47B10981159940AD43B10523
:1033400020F48CE085B98EE15AC0D701C6019B51AB
:10335000A74BB10981159940AD43B10520F480E137
:1033600085B984E14CC0D701C6019452A44FB1097C
:10337000803C964CAD42B10520F484E185B981E1F1
:103380003EC0D701C601805C9A4EA142B140803C4C
:10339000964CAD42B10520F488E185B98FE02FC08D
:1033A000D701C6018058914BAF44B14080349B4453
:1033B000AC44B10520F48CE185B98CE020C0D70184
:1033C000C601805C9C4FAB49B14080349D45A64C02
:1033D000B10520F480E285B98AE011C08AE5D81AE7
:1033E00082E6E80A82E0F80A91E4C9169DE5D9066A
:1033F00096ECE906F10428F484E285B986E080932E
:10340000860260E070E0CB010E9443058091640277
:1034100090916502009729F481E090E0A0E0B0E08F
:103420006CC08130910529F48AE090E0A0E0B0E022
:1034300064C0883EA3E09A0749F440924E0250923D
:103440004F0260925002709251025FC08A30910523
:1034500029F484E690E0A0E0B0E04FC0893EA3E00C
:103460009A0729F48AEF90E0A0E0B0E046C0823FDE
:10347000A3E09A0729F484EF91E0A0E0B0E03DC01A
:103480008B30910529F488EE93E0A0E0B0E035C0E0
:10349000833FB3E09B0729F488E893E1A0E0B0E024
:1034A0002CC08C34A4E09A0729F488E293E2A0E0CF
:1034B000B0E023C08436910529F480E197E2A0E0D2
:1034C000B0E01BC08536910529F480EA96E8A1E0BA
:1034D000B0E013C08E36910549F480924E0290926E
:1034E0004F02A0925002B09251020FC08F36910548
:1034F00061F480E896E9A8E9B0E080934E029093E9
:103500004F02A0935002B093510260E070E0CB01F3
:103510000E9443050E9472110E9472117C016AE0B0
:1035200070E080E090E00E9443050E9472110E94CA
:103530007211092E000CAA0BBB0BA7010F2C000C5B
:10354000660B770B8C019D010D5F1F4F2F4F3F4F77
:10355000041715072607370764F00397A109B10977
:10356000481759076A077B0724F0F0926A02E09235
:1035700069028091690290916A028538A3E09A07F6
:103580005CF0109268021092670210927C02109216
:103590005A02109266029CC08C30910554F420911E
:1035A0006802213031F01092680281E080937C0241
:1035B0008FC09C01235331092D31310550F42091E6
:1035C0006802211103C068E871E00FC0213009F4DE
:1035D0007FC09C01205631092C323105A8F420917E
:1035E000680221110EC06EE871E08DE493E00E9444
:1035F000670481E0809368026EE170E080E090E013
:1036000065C0213009F464C09C012C593109223273
:10361000310550F420916802211103C064E971E082
:103620000FC0213009F454C09C01295C31092D31AF
:10363000310580F42091680221110AC068E971E027
:103640008DE493E00E94670481E0809368023AC0B1
:103650002130F1F19C01215F31092D31310560F4F8
:1036600020916802211106C081E080936802809356
:10367000660228C0213061F19C012951314023317B
:10368000310530F420916802222371F3213001F1D9
:103690009C01275331402732310530F420916802D4
:1036A000222311F32130A1F08159914085399105F0
:1036B00078F48091680281110BC081E080936802E8
:1036C00080935A0268E270E080E090E00E94430537
:1036D00060E070E0CB010E94430510917C02113044
:1036E00081F480916B02813061F061E081E10E94A0
:1036F000C1046CE971E08DE493E00E9467041093CB
:103700006B0280917C02811110C080916B0281302C
:1037100061F460E081E10E94C10460EA71E08DE43F
:1037200093E00E94670410926B0210918A0211309C
:1037300011F461E003C0111104C060E081E10E9456
:10374000C10480918B028F5F80938B02843109F0DA
:103750008BC0113009F488C010928B0264EA71E0CA
:103760008DE493E00E9467048DE493E00E94690178
:1037700068E270E080E090E00E9443058DE493E011
:103780000E94EB00181619060CF062C08DE493E05D
:103790000E94C900809372028A3531F080917102D3
:1037A000882309F455C019C08AE50E94411501E03B
:1037B0008DE493E00E94EB00181619067CF78DE467
:1037C00093E00E94C900182F809372020E94411555
:1037D0001B3371F700937102EBCF60E874E084E46F
:1037E00094E00E94DB0325E030E044E050E064E434
:1037F00074E0CE0101960E940C04BE016F5F7F4F02
:103800008EE394E00E940303CE0101960E94F2032E
:103810008EE394E00E94F80260937B02611102C083
:1038200061E003C0613031F460E08FE00E94C104C8
:1038300060E00BC0623011F461E003C0633041F41A
:1038400060E08FE00E94C10461E080E10E94C10459
:1038500067E871E084E494E00E94C40367E871E0E3
:1038600080E894E00E94C403809189028F5F809376
:1038700089028A3009F079C080918A02813009F486
:1038800074C0109289026AEA71E08DE493E00E94AC
:1038900067048DE493E00E94690168E270E080E0D3
:1038A00090E00E9443058DE493E00E94EB0018161F
:1038B00019060CF04EC08DE493E00E94C90080937D
:1038C00072028A3569F180917102882309F441C03E
:1038D00060E874E088E394E00E94DB0328E030E0D5
:1038E00045E050E068E374E0CE0101960E940C04CC
:1038F000BE016F5F7F4F82E394E00E940303CE011D
:1039000001960E94F20382E394E00E94F802609321
:10391000730270937402809375029093760219C0BB
:103920008AE50E94411501E08DE493E00E94EB00DE
:103930001816190644F68DE493E00E94C900182F6A
:10394000809372020E9441151B3371F7009371023C
:10395000EBCF67E871E088E394E00E94C40367E876
:1039600071E080E894E00E94C403809188028F5F38
:1039700080938802843109F074C01092880261EB50
:1039800071E08DE493E00E9467048DE493E00E946F
:10399000690168E270E080E090E00E9443058DE4F8
:1039A00093E00E94EB00181619060CF04EC08DE44F
:1039B00093E00E94C900809372028A3531F08091B1
:1039C0007102882309F441C019C08AE50E9441159B
:1039D00001E08DE493E00E94EB00181619067CF7D5
:1039E0008DE493E00E94C900182F809372020E9418
:1039F00041151B3371F700937102EBCF60E874E05F
:103A000084E194E00E94DB0325E030E044E050E0F4
:103A100064E174E0CE0101960E940C04BE016F5F68
:103A20007F4F8EE094E00E940303CE0101960E9436
:103A3000F2038EE094E00E94F80260936C02613021
:103A400009F060E084E10E94C10467E871E084E16C
:103A500094E00E94C40367E871E080E894E00E946B
:103A6000C40380918A02813009F072C067EB71E073
:103A70008DE493E00E9467048DE493E00E94690165
:103A800068E270E080E090E00E9443058DE493E0FE
:103A90000E94EB00181619060CF04EC08DE493E05E
:103AA0000E94C90080937202863469F1809171028C
:103AB000882309F441C060E874E080E294E00E9449
:103AC000DB032DE030E044E050E060E274E0CE0142
:103AD00001960E940C04BE016F5F7F4F8AE194E063
:103AE0000E940303CE0101960E94F2038AE194E052
:103AF0000E94F80260936D0270936E0280936F02D1
:103B00009093700219C086E40E94411501E08DE493
:103B100093E00E94EB001816190644F68DE493E03A
:103B20000E94C900182F809372020E9441151B3316
:103B300071F700937102EBCF67E871E080E294E0E7
:103B40000E94C40367E871E080E894E00E94C40327
:103B500080915A0260E0813009F463C383E00E94DF
:103B60000C1560910001709101018091020190910A
:103B70000301A50194010E9446252A30310558F41D
:103B800080E22FA738AB49AB5AAB0E94C8115AA9A3
:103B900049A938A92FA5CA01B901882799274AE060
:103BA0000E9485118EE20E94C811609100017091FF
:103BB00001018091020190910301A50194010E94ED
:103BC000462528EE33E040E050E00E94462589017A
:103BD00024363105A8F480E32FA738AB49AB5AABA4
:103BE0000E94C8112FA538A949A95AA90A30110560
:103BF00038F480E30E94C8115AA949A938A92FA511
:103C0000CA01B901882799274AE00E9485118EE2EE
:103C10000E94C81160910001709101018091020120
:103C20009091030128EE33E040E050E00E944625E9
:103C30006B017C018B016436710548F480E30E94BE
:103C4000C8110A30110518F480E30E94C811C70199
:103C5000B601882799274AE00E9485116BEB71E035
:103C600086EF93E00E94670480917C0281110DC071
:103C700080918A02811109C060E00E940C156FEBEF
:103C800071E086EF93E00E94670480917C028130AE
:103C900021F080918A02813081F465E871E086EF3D
:103CA00093E00E94670460E080E00E940C1563ECE2
:103CB00071E086EF93E00E94670461E084E00E9477
:103CC0000C1564E871E086EF93E00E946704809130
:103CD0007B02811109C061E00E940C1567EC71E064
:103CE00086EF93E00E94670480917B02813051F45B
:103CF00061E080E00E940C156CEC71E086EF93E0CF
:103D00000E94670480917B02823051F461E080E080
:103D10000E940C1561ED71E086EF93E00E9467044C
:103D200080917B02833051F461E080E00E940C15A9
:103D300066ED71E086EF93E00E9467042FB7F89478
:103D40008091520290915302A0915402B091550279
:103D50002FBF409177025091780260917902709163
:103D60007A02841B950BA60BB70B853F9140A105EA
:103D7000B10508F488C261E087E00E940C156BED84
:103D800071E086EF93E00E94670480917302909146
:103D90007402A0917502B091760281319105A1055E
:103DA000B105BCF464E871E086EF93E00E9467041B
:103DB00061E08AE00E940C1564E871E086EF93E010
:103DC0000E94670461E08AE00E940C156FED71E0CB
:103DD00010C2AC01BD01405151096109710947315F
:103DE00051056105710588F461E08AE00E940C15B7
:103DF00061E871E086EF93E00E94670461E08AE089
:103E00000E940C1561EE71E0F4C1AC01BD01475296
:103E1000510961097109413151056105710588F444
:103E200061E08AE00E940C1561E871E086EF93E0A2
:103E30000E94670461E08AE00E940C1563EE71E065
:103E4000D8C1AC01BD0148535109610971094A301B
:103E500051056105710588F461E08AE00E940C1546
:103E600061E871E086EF93E00E94670461E08AE018
:103E70000E940C1565EE71E0BCC1AC01BD0142545D
:103E80005109610971094A3051056105710588F4CC
:103E900061E08AE00E940C1561E871E086EF93E032
:103EA0000E94670461E08AE00E940C1567EE71E0F1
:103EB000A0C1AC01BD014C545109610971094F30D9
:103EC00051056105710588F461E08AE00E940C15D6
:103ED00061E871E086EF93E00E94670461E08AE0A8
:103EE0000E940C1569EE71E084C1AC01BD014B5517
:103EF0005109610971094A3051056105710588F45C
:103F000061E08AE00E940C1561E871E086EF93E0C1
:103F10000E94670461E08AE00E940C156BEE71E07C
:103F200068C1AC01BD0145565109610971094F30A5
:103F300051056105710588F461E08AE00E940C1565
:103F400061E871E086EF93E00E94670461E08AE037
:103F50000E940C156DEE71E04CC1AC01BD014457DF
:103F60005109610971094D3051056105710588F4E8
:103F700061E08AE00E940C1561E871E086EF93E051
:103F80000E94670461E08AE00E940C156FEE71E008
:103F900030C1AC01BD014158510961097109473077
:103FA00051056105710588F461E08AE00E940C15F5
:103FB00061E871E086EF93E00E94670461E08AE0C7
:103FC0000E940C1561EF71E014C1AC01BD014858AD
:103FD0005109610971094F3051056105710588F476
:103FE00061E08AE00E940C1561E871E086EF93E0E1
:103FF0000E94670461E08AE00E940C1563EF71E0A3
:10400000F8C0AC01BD0147595109610971094F3030
:1040100051056105710588F461E08AE00E940C1584
:1040200061E871E086EF93E00E94670461E08AE056
:104030000E940C156AEF71E0DCC0AC01BD01465A6C
:104040005109610971094F3051056105710588F405
:1040500061E08AE00E940C1561E871E086EF93E070
:104060000E94670461E08AE00E940C1561E072E042
:10407000C0C0AC01BD01455B5109610971094A30FD
:1040800051056105710588F461E08AE00E940C1514
:1040900061E871E086EF93E00E94670461E08AE0E6
:1040A0000E940C1568E072E0A4C0AC01BD014F5B3A
:1040B0005109610971094A3051056105710588F49A
:1040C00061E08AE00E940C1561E871E086EF93E000
:1040D0000E94670461E08AE00E940C156FE072E0C4
:1040E00088C0AC01BD01495C5109610971094A30C0
:1040F00051056105710588F461E08AE00E940C15A4
:1041000061E871E086EF93E00E94670461E08AE075
:104110000E940C1566E172E06CC0AC01BD01435D0C
:104120005109610971094F3051056105710588F424
:1041300061E08AE00E940C1561E871E086EF93E08F
:104140000E94670461E08AE00E940C156DE172E054
:1041500050C0AC01BD01425E5109610971094F3087
:1041600051056105710588F461E08AE00E940C1533
:1041700061E871E086EF93E00E94670461E08AE005
:104180000E940C1564E272E034C0AC01BD01415FD5
:104190005109610971094A3051056105710588F4B9
:1041A00061E08AE00E940C1561E871E086EF93E01F
:1041B0000E94670461E08AE00E940C156BE272E0E5
:1041C00018C08B5F9109A109B1090A97A105B10532
:1041D000A0F461E08AE00E940C1561E871E086EFCE
:1041E00093E00E94670461E08AE00E940C1562E39C
:1041F00072E086EF93E00E9467042FB7F8948091F5
:10420000520290915302A0915402B09155022FBFD7
:104210008093770290937802A0937902B0937A0208
:1042200032C080E00E940C1569E372E086EF93E0F3
:104230000E94670461E080E00E940C1568E771E06D
:1042400086EF93E00E94670461E085E00E940C1510
:10425000C0905602D0905702E0905802F090590258
:10426000F7FE0CC08DE20E94C81166277727CB01AC
:104270006C197D098E099F094AE003C04AE0C70115
:10428000B6010E9485118091000190910101A091D9
:104290000201B091030181349244AF40B10544F46E
:1042A0008092000190920101A0920201B09203015C
:1042B0008091000190910101A0910201B091030150
:1042C000803C9243AA40B34064F080EC92E3AAE0C1
:1042D000B3E08093000190930101A0930201B09399
:1042E00003019091830280918A029430B9F4813065
:1042F000A9F48091000190910101A0910201B09177
:104300000301885F9A42A109B1098093000190934B
:104310000101A0930201B093030123C081111EC0CB
:1043200080918202811105C0809181028111C8C0F3
:1043300008C0813009F062C080918102813009F0AB
:10434000C3C08091000190910101A0910201B09140
:10435000030188529342A109B10948C0813009F094
:104360004DC080918202811149C0809181028130CB
:1043700009F044C08AE492E00E9421158823E1F00C
:10438000409100015091010160910201709103017F
:1043900080917D0290917E02A0917F02B091800277
:1043A000840F951FA61FB71F8093000190930101F2
:1043B000A0930201B09303018CE492E00E942115C6
:1043C0008823E1F08091000190910101A091020108
:1043D000B091030140917D0250917E0260917F0275
:1043E00070918002841B950BA60BB70B8093000184
:1043F00090930101A0930201B09303018091870281
:104400008F5F883C19F08093870202C01092870268
:10441000C0900001D0900101E0900201F0900301F2
:1044200080918C0290918D02A0918E02B0918F02AA
:10443000C816D906EA06FB0699F0C701B60122E0C4
:10444000660F771F881F991F2A95D1F724E630E061
:1044500040E050E00E94C42500E010E00E94290DD9
:1044600030908602809185023816C1F080918402D6
:10447000811114C0C701B601685B7E488F4F9F4F02
:1044800024E630E040E050E00E94C42502E010E065
:104490000E94290D3092850210928702C0928C02F0
:1044A000D0928D02E0928E02F0928F020E948B01D8
:1044B0000C94DB16CE0101960E9491030C946F17A9
:1044C000813009F09BCF3DCF811198CFC090000182
:1044D000D0900101E0900201F090030188E2C81A37
:1044E00083E2D80AE108F108C0920001D0920101EC
:1044F000E0920201F09203018AE492E00E94211509
:10450000882309F459CF80917D0290917E02A09179
:104510007F02B0918002C80ED91EEA1EFB1EC09217
:104520000001D0920101E0920201F092030144CF18
:104530008EE094E00E94F20384E194E00E94F20392
:104540008AE194E00E94F20380E294E00E94F20388
:1045500086E294E00E94F2038CE294E00E94F2036F
:1045600082E394E00E94F20388E394E00E94F20365
:104570008EE394E00E94F20384E494E00E94F2034C
:104580008AE494E00E94F20380E594E00E94F20342
:1045900086E594E00E94F2038CE594E00E94F20329
:1045A00082E694E00E94F20388E694E00E94F2031F
:1045B0008EE694E00E94F20384E794E00E94F20306
:1045C0008AE794E00E94F20380E894E00C94F203FE
:1045D0001F93CF93DF93EDE4F3E01382128288EE12
:1045E00093E0A0E0B0E084839583A683B7832AE2BA
:1045F00031E03183208325EC30E03587248724ECBB
:1046000030E03787268720EC30E0318B208B21EC9F
:1046100030E0338B228B22EC30E0358B248B26EC80
:1046200030E0378B268B118E128E138E148EEAEEAD
:10463000F3E01382128284839583A683B7838AE38F
:1046400091E091838083E9E8F4E018E010AF11AFC6
:1046500011AA12AA13AA1186128613861486158629
:1046600016861786108A118A128A138A148A158A66
:10467000168A178A108E118E128E138E148E158E36
:10468000168E178E10A211A212A213A214A215A2A6
:1046900016A217A210A611A612A613A614A615A656
:1046A00016A617A610AA80E098E4A8EEB1E082AFA3
:1046B00093AFA4AFB5AFC6E8D4E082E0898383E0CE
:1046C0008A8360E082E00E94070560E08A810E94A0
:1046D000070561E089810E94C10461E08A810E942E
:1046E000C104188267E871E080E894E00E94F70353
:1046F00067E871E08AE794E00E94F70367E871E0F9
:1047000084E794E00E94F70367E871E08EE694E0A6
:104710000E94F70367E871E088E694E00E94F703DF
:1047200067E871E082E694E00E94F70367E871E0D1
:104730008CE594E00E94F70367E871E086E594E079
:104740000E94F70367E871E080E594E00E94F703B8
:1047500067E871E08AE494E00E94F70367E871E09B
:1047600084E494E00E94F70367E871E08EE394E04C
:104770000E94F70367E871E088E394E00E94F70382
:1047800067E871E082E394E00E94F70367E871E074
:104790008CE294E00E94F70367E871E086E294E01F
:1047A0000E94F70367E871E080E294E00E94F7035B
:1047B00067E871E08AE194E00E94F70367E871E03E
:1047C00084E194E00E94F70367E871E08EE094E0F2
:1047D0000E94F703E6EFF3E0138212828AE491E08D
:1047E0009183808389E084838FEF8583168387E0BC
:1047F000878386E0808785E0818784E082871386CF
:10480000148615861686178661E0CF01DF91CF9159
:104810001F910C94D3111F93FC0199278827BC0189
:10482000E89411911032E9F3193010F01E30C8F3FA
:104830001B3251F01D3249F4689406C00E944C248A
:10484000610F711D811D911D119110531A30B0F32C
:104850003EF490958095709561957F4F8F4F9F4F57
:104860001F910895BB274A3031F4992322F4BDE209
:10487000909581959F4F0C948424BB272A3051F446
:10488000992342F4BDE290958095709561957F4F94
:104890008F4F9F4F0C946224592F482F372F262F6C
:1048A000660F771F881F991F660F771F881F991F34
:1048B000620F731F841F951F660F771F881F991F34
:1048C0000895BB27FA01A62F62177105810591058E
:1048D000330B30FB66F0AA27660F771F881F991FDE
:1048E000AA1FA21710F0A21B63953850A9F7A05D6C
:1048F000AA3308F0A95DA19336F7B111B1931082E4
:10490000CA010C949D24BB27FB015527AA27880FB9
:10491000991FAA1FA41710F0A41B83955051B9F733
:10492000A05DAA3308F0A95DA193009779F7B111B2
:10493000B1931192CB010C949D24DC01FC01672FF3
:1049400071917723E1F7329704C07C916D93708366
:104950006291AE17BF07C8F30895F999FECF92BDD3
:1049600081BDF89A992780B50895262FF999FECF31
:104970001FBA92BD81BD20BD0FB6F894FA9AF99A7C
:104980000FBE019608950E940525A59F900DB49F26
:10499000900DA49F800D911D112408952F923F9298
:1049A0004F925F926F927F928F929F92AF92BF923F
:1049B000CF92DF92EF92FF920F931F93CF93DF93EB
:1049C000CDB7DEB7CA1BDB0B0FB6F894DEBF0FBE48
:1049D000CDBF09942A88398848885F846E847D8495
:1049E0008C849B84AA84B984C884DF80EE80FD8097
:1049F0000C811B81AA81B981CE0FD11D0FB6F8940D
:104A0000DEBF0FBECDBFED010895A29FB001B39FE1
:104A1000C001A39F700D811D1124911DB29F700DC7
:104A2000811D1124911D0895DB018F939F930E9496
:104A3000C324BF91AF91A29F800D911DA39F900DA4
:104A4000B29F900D11240895A1E21A2EAA1BBB1B40
:104A5000FD010DC0AA1FBB1FEE1FFF1FA217B3074A
:104A6000E407F50720F0A21BB30BE40BF50B661F60
:104A7000771F881F991F1A9469F760957095809524
:104A800090959B01AC01BD01CF010895052E97FBC8
:104A90001EF400940E945D2557FD07D00E94242536
:104AA00007FC03D04EF40C945D255095409530954D
:104AB00021953F4F4F4F5F4F08959095809570958A
:104AC00061957F4F8F4F9F4F0895EE0FFF1F059009
:104AD000F491E02D0994DF93CF931F930F939A9D48
:104AE000F02D219FF00D8B9DF00D8A9DE02DF10D95
:104AF000039FF00D029FE00DF11D4E9DE00DF11D95
:104B00005E9DF00D4F9DF00D7F936F93BF92AF921E
:104B10005F934F93D5010E9405258B01AC01D7010E
:104B20000E940525EB01E80FF91FD6010E94BB2565
:104B30002F913F91D6010E940525C60FD71FE81F70
:104B4000F91FAF91BF910E94BB252F913F910E9409
:104B50000525C60FD71FE81FF91FD6010E9405259E
:104B6000E60FF71F9801BE01CF0111240F911F918D
:104B7000CF91DF9108950E940525460F571FC81F4A
:104B8000D91F08F43196089597FB57FF0C94D4254C
:104B90009F938F930E94D4256E1B7F0BAF91BF9183
:104BA0008A0B9B0B0895E894DF93CF93FC01DB0104
:104BB0000E9405257F936F93E9019A01AC01BF9391
:104BC000AF933F932F93DF010E94052526F46C1BC2
:104BD0007D0B820B930B9E01EB01FC010E94BB2518
:104BE000AF91BF912F913F910E94BB25BE01CF0194
:104BF000F9012F913F91CF91DF910895689401C001
:104C0000E894F92FF12B12F00C943226A0E0B0E0DA
:104C1000ECE0F6E20C94D424092E059422F40E94D0
:104C20008E26112392F4F0E80F26FFEFE094F09423
:104C300000951095B094C094D094A194BF0ACF0A67
:104C4000DF0AEF0AFF0A0F0B1F0B0E943D2607FC2D
:104C50000E948E26CDB7DEB7ECE00C94F024689469
:104C600001C0E8948F929F92CF93DF930E943D26DC
:104C7000DF91CF919F908F90089588249924F4011B
:104C8000E401B0E49F93AA279A158B049C04ED05D8
:104C9000FE05CF05D007A10798F4AD2FDC2FCF2F4D
:104CA000FE2FE92D982C892E982F872F762F652F90
:104CB000542F432F322F2227B85031F7BF9127C0EE
:104CC0001B2EBF91BB27220F331F441F551F661F8A
:104CD000771F881F991F881C991CEE1FFF1FCC1F70
:104CE000DD1FAA1FBB1F8A149B04EC05FD05CE0522
:104CF000DF05A007B10748F08A189B08EC09FD09F9
:104D0000CE09DF09A00BB10B21601A94E1F62EF455
:104D10009401AF01BE01CD01000C0895609570951E
:104D20008095909530954095509521953F4F4F4FE8
:104D30005F4F6F4F7F4F8F4F9F4F08950F930830F6
:104D400090F0982F872F762F652F542F432F322FD7
:104D500022270850F4CF220F331F441F551F661F10
:104D6000771F881F991F0A95B2F70F91089597FB37
:104D700010F8169400080F93083098F00850232F6D
:104D8000342F452F562F672F782F892F902DF4CF52
:104D90000594979587957795679557954795379596
:104DA00027950A95AAF70F9108952A0D3B1D4C1DD2
:104DB0005D1D6E1D7F1D801F911F08952A193B09DF
:104DC0004C095D096E097F09800B910B08952A1526
:104DD0003B054C055D056E057F058007910708952D
:104DE0000024A7FD00942A173005400550056005F2
:104DF0007005800590050895CF93DF93823091056B
:104E000010F482E090E0E091C904F091CA0420E03F
:104E100030E0C0E0D0E0309711F140815181481777
:104E20005907C0F04817590761F482819381209790
:104E300019F09B838A832BC09093CA048093C90482
:104E400026C02115310519F04217530718F49A01AD
:104E5000BE01DF01EF010280F381E02DDCCF2115DF
:104E6000310509F1281B390B2430310590F41296D5
:104E70008D919C9113976115710521F0FB0193832E
:104E8000828304C09093CA048093C904FD013296C2
:104E900044C0FD01E20FF31F819391932250310929
:104EA0002D933C933AC02091C7043091C804232B22
:104EB00041F420910601309107013093C8042093FA
:104EC000C70420910401309105012115310541F4F9
:104ED0002DB73EB74091080150910901241B350BB5
:104EE000E091C704F091C804E217F307A0F42E1B69
:104EF0003F0B2817390778F0AC014E5F5F4F24173E
:104F0000350748F04E0F5F1F5093C8044093C70405
:104F10008193919302C0E0E0F0E0CF01DF91CF9167
:104F200008950F931F93CF93DF93009709F48CC0DC
:104F3000FC013297138212820091C9041091CA04B5
:104F40000115110581F420813181820F931F209179
:104F5000C7043091C8042817390779F5F093C804BD
:104F6000E093C70471C0D80140E050E0AE17BF071E
:104F700050F412962D913C911397AD0121153105F6
:104F800009F1D901F3CF9D01DA01338322836081D6
:104F90007181860F971F8217930769F4EC012881AE
:104FA0003981260F371F2E5F3F4F318320838A813F
:104FB0009B8193838283452B29F4F093CA04E09369
:104FC000C90442C01396FC93EE931297ED014991E8
:104FD00059919E01240F351FE217F30771F4808168
:104FE0009181840F951F029611969C938E938281D6
:104FF000938113969C938E931297E0E0F0E0D80192
:1050000012968D919C911397009719F0F8018C01DD
:10501000F6CF8D919C9198012E5F3F4F820F931F89
:105020002091C7043091C8042817390769F43097D4
:1050300029F41092CA041092C90402C01382128289
:105040001093C8040093C704DF91CF911F910F9173
:105050000895A0E0B0E0EFE2F8E20C94D224EC0175
:10506000009721F4CB010E94FC26B8C0FC01E60F9A
:10507000F71F9C0122503109E217F30708F4ACC076
:10508000D9010D911C91119706171707B0F0053043
:10509000110508F49FC0C80104978617970708F404
:1050A00099C002501109061B170B019311936D93C0
:1050B0007C93CF010E9491278DC05B01A01AB10A99
:1050C0004C01800E911EA091C904B091CA0440E029
:1050D00050E0E12CF12C109709F44AC0A815B9054D
:1050E000D1F56D907C901197630182E0C80ED11CC0
:1050F000CA14DB0480F1A3014A195B096A0182E04A
:10510000C80ED11C1296BC9012971396AC91B5E0C4
:10511000CB16D10440F0B282A38351834083D901DE
:105120006D937C930AC00E5F1F4FC301800F911FC8
:10513000F90191838083EB2DFA2FE114F10431F012
:10514000D7011396FC93EE93129744C0F093CA04D0
:10515000E093C9043FC08D919C911197481759075E
:1051600008F4AC017D0112960D90BC91A02DB3CF37
:105170008091C7049091C80488159905E1F44617F9
:105180005707C8F48091040190910501009741F4FC
:105190008DB79EB74091080150910901841B950B72
:1051A000E817F907C8F4F093C804E093C704F901BD
:1051B000718360830FC0CB010E94FC267C010097A5
:1051C00059F0A801BE010E94F828CE010E94912743
:1051D000C70104C0CE0102C080E090E0CDB7DEB7C9
:1051E000EEE00C94EE2481E090E0F8940C94112908
:1051F000FB01DC0102C001900D9241505040D8F7F4
:105200000895FB01DC018D91019080190110D9F303
:10521000990B0895FB01DC0101900D920020E1F74C
:10522000089510E0C2E7D0E004C0FE010E946525A9
:0C5230002196C337D107C9F7F894FFCFCF
:10523C00D0B137000000CB04800000020400030052
:10524C000110030200000302010006000400060521
:10525C000020060504000000000022019E00EB0067
:10526C00C900DD006901000000009A026A026202B6
:10527C004E023F023E020000000075079E004641B0
:10528C000049463B0020204E6F20636F6E6E6563B5
:10529C0074696F6E200020202020506F7765725348
:1052AC0044522020202000202020202020202020BC
:1052BC0020202020202020005A5A53553B005A5AB7
:1052CC0053443B0042553B0042443B0054583B0086
:1052DC0052583B005A5A50413B005A5A534D303B9E
:1052EC00005A5A4D4F3B0046423B0020487A005230
:1052FC00582000545820004F666620004C6F7720D1
:10530C00004D656420004869676800536D3A0030B1
:10531C0000310032003300340035003600370038DD
:10532C00003900392B2035644200392B313064426E
:10533C0000392B3230644200392B3235644200394B
:10534C002B3330644200392B3335644200392B3413
:10535C0030644200392B3530644200392B363064CE
:10536C004200392B3730644200436F7272656374AC
:0E537C00696F6E202046524551002B002D0017
:00000001FF
